:100000000C9434000C9451000C9451000C94510049
:100010000C9451000C9451000C9451000C9451001C
:100020000C9451000C9451000C9451000C9451000C
:100030000C9451000C9451000C9451000C945100FC
:100040000C9467000C9451000C9451000C945100D6
:100050000C9451000C9451000C9451000C945100DC
:100060000C9451000C94510011241FBECFEFD8E026
:10007000DEBFCDBF11E0A0E0B1E0E8EDF1E002C0ED
:1000800005900D92A030B107D9F711E0A0E0B1E0E2
:1000900001C01D92A930B107E1F70E9456000C94EF
:1000A000EA000C940000089508950895CF93DF931B
:1000B0000E94AF000E9455000E945300C0E0D0E0B3
:1000C0000E9454002097E1F30E940000F9CF1F9294
:1000D0000F920FB60F9211242F933F938F939F93FC
:1000E000AF93BF938091040190910501A091060107
:1000F000B0910701309108010196A11DB11D232F78
:100100002D5F2D3720F02D570196A11DB11D209395
:1001100008018093040190930501A0930601B09318
:1001200007018091000190910101A0910201B0911D
:1001300003010196A11DB11D80930001909301015F
:10014000A0930201B0930301BF91AF919F918F9152
:100150003F912F910F900FBE0F901F90189578949C
:1001600084B5826084BD84B5816084BD85B58260BC
:1001700085BD85B5816085BDEEE6F0E0808181605A
:100180008083E1E8F0E0108280818260808380815A
:1001900081608083E0E8F0E0808181608083E1EB32
:1001A000F0E0808184608083E0EBF0E0808181601A
:1001B0008083EAE7F0E080818460808380818260D0
:1001C00080838081816080838081806880831092B9
:0801D000C1000895F894FFCF6F
:00000001FF
